:0200000480007A
:100000006F00C0006F20C0276F2080279300000082
:10001000130100009301000013020000930200008E
:100020001303000093030000130400009304000076
:10003000130500009305000013060000930600005E
:100040001307000093070000130800009308000046
:100050001309000093090000130A0000930A00002E
:10006000130B0000930B0000130C0000930C000016
:10007000130D0000930D0000130E0000930E0000FE
:10008000130F0000930F000097020000938202F804
:1000900073905230177100001301412DF32240F18B
:1000A0009392C2003301510073100134EF20103AD3
:1000B00017350000130505BA6F20D01583224508B7
:1000C0007390121483204500032185008321C5000D
:1000D0000322050183224501032385018323C501F2
:1000E00003240502832445028325C5020326050354
:1000F00083264503032785038327C50303280504B7
:1001000083284504032985048329C504032A05059A
:10011000832A4505032B8505832BC505032C05067E
:10012000832C4506032D8506832DC506032E050762
:10013000832E4507032F8507832FC50703258502D7
:1001400073002010731101142322110023263100A3
:1001500023284100232A5100232C6100232E710003
:1001600023208102232291022324A1022326B1020B
:100170002328C102232AD102232CE102232EF102DB
:1001800023200105232211052324210523263105DF
:1001900023284105232A5105232C6105232E7105AF
:1001A00023208107232291072324A1072326B107B7
:1001B0002328C107232AD107232CE107232EF10787
:1001C000F312011423245100F322001023205108BC
:1001D000F322101423225108F3223014232451084F
:1001E000F322201423265108130501006F20004735
:1010000000000000000000000000000000000000E0
:1010100000000000000000000000000000000000D0
:1010200000000000000000000000000000000000C0
:1010300000000000000000000000000000000000B0
:081040000000000000000000A8
:10200000B3E7C500B367F50093F73700B306C50023
:10201000638407023386C50093070500637ED502FB
:1020200003C705009385150093871700A38FE7FE6C
:10203000E398C5FE67800000E37ED5FE93070500A8
:1020400003A70500938747009385450023AEE7FE6D
:10205000E3E8D7FE6780000067800000B367C50033
:1020600093F737003306C5006380070293F5F50F39
:10207000930705006370C50493871700A38FB7FE0D
:10208000E31CF6FE6780000093F5F50F939785003B
:10209000B3E7B70093950701B3E5F500E374C5FE18
:1020A000930705009387470023AEB7FEE3ECC7FE16
:1020B000678000006780000083470500638E07008B
:1020C0009307050003C7170093871700E31C07FE5B
:1020D0003385A7406780000013050000678000007B
:1020E00083470500938515001305150003C7F5FF09
:1020F00063880700E386E7FE3385E74067800000DA
:10210000930700006FF05FFFB367B50093F73700E8
:10211000639E07021378C6FF330805016378050341
:10212000930705006F0000019387470093854500E2
:1021300063F8070183A6070003A70500E386E6FE10
:102140003385A7403306A640138507003386C500B4
:102150006F00400103C705008347F5FF9385150015
:10216000639AE70013051500E396C5FE130500000A
:10217000678000003385E740678000009307050013
:1021800003C705009387170093851500A38FE7FE0B
:10219000E31807FE6780000003470500930600026E
:1021A000930705006318D70003C71700938717002C
:1021B000E30CD7FE9306D0026300D7069306B00265
:1021C0006300D70483C607009305000063820604FA
:1021D0001305000093871700138606FD13172500CB
:1021E00083C607003305A700131515003305A600A5
:1021F000E39206FE638005023305A040678000007D
:1022000083C617009305000093871700E39206FC2E
:10221000130500006780000083C6170093051000B7
:1022200093871700E39606FA130500006FF09FFEF0
:1022300017F6FFFF130606DD032706008327460077
:102240009355F5413367F7006306070297F6FFFFE2
:10225000938646DF9307000023A0F60013080000D2
:1022600023A2060103270600832746003367F700F1
:10227000E31207FE2320A6002322B6006F00000011
:10228000130101FF1305903423261100EFF05FFACC
:10229000130101FE1306C1001307B10113039000DF
:1022A0006F008000138707009377F500B337F300C2
:1022B000B307F04093F777029376F500938707030F
:1022C000B387F6002300F7009396C5011355450028
:1022D0009307F7FF33E5A60093D54500E314E6FC2A
:1022E0000345C100230E01006302050693050600A5
:1022F00097F6FFFF938606D117F6FFFF130686D4E5
:1023000003A7060083A74600130805009385150060
:102310003367F700B70801016302070213070000E3
:102320002320E600930700002322F60003A70600FF
:1023300083A746003367F700E31207FE03C50500D5
:1023400023A0060123A21601E31C05FA13010102D2
:102350006780000037F6FFFF3307C500B7E70300CB
:102360006370F7149356C50093820640172300004C
:10237000130343C993972200B307F30003A7070091
:102380003375C5006306070293760704638C060E57
:1023900093760708639206189306F000639ED5169D
:1023A0001367070823A0E700730005126780000089
:1023B0001747000013074704832507006384051CA3
:1023C00083A74500174600000326C6022320F70016
:1023D0006382C70C03A7050093972200B307F3009D
:1023E0001357C7001317A700136EF70D1366F701F5
:1023F00023A0C7017300051297470000938707E0E9
:1024000093963600B386D70083A706006392071E13
:1024100083A7050023A0F60083A74500B7050400A5
:1024200023A2F600F3A50510B707C0FFB307F50018
:10243000B716000013070500B386D70083AE070068
:1024400003AE470083A8870003A8C7002320D70155
:102450002322C7012324170123260701938707019D
:1024600013070701E39CD7FC739005109397220094
:10247000B307F30023A0C700730005120F1000007C
:10248000678000001367070423A0E70073000512AC
:10249000678000009747000023AE07F46FF09FF3BA
:1024A0001305100497150000938585CA97F6FFFF62
:1024B000938646B517F6FFFF1306C6B803A70600B6
:1024C00083A7460013030500938515003367F700C3
:1024D000B703010163020702930700002320F600FF
:1024E000130800002322060103A7060083A7460065
:1024F0003367F700E31207FE03C5050023A066005B
:1025000023A27600E31C05FA130101FF1305300036
:1025100023261100EFF0DFD11305100497150000FA
:10252000938545C797F6FFFF9386C6AD17F6FFFF65
:10253000130646B103A7060083A74600130E050045
:10254000938515003367F700B70E01016302070298
:10255000930700002320F600130800002322060141
:1025600003A7060083A746003367F700E31207FEC0
:1025700003C5050023A0C60123A2D601E31C05FA6A
:102580006FF09FF81305100497150000938505C59B
:1025900097F6FFFF938606A717F6FFFF130686AA96
:1025A00003A7060083A74600130F050093851500B7
:1025B0003367F700B70F01016302070293070000BA
:1025C0002320F600130800002322060103A70600BB
:1025D00083A746003367F700E31207FE03C5050033
:1025E00023A0E60123A2F601E31C05FA6FF0DFF158
:1025F00013051004971500009385C5BF97F6FFFFDC
:10260000938646A017F6FFFF1306C6A303A706008E
:1026100083A7460013080500938515003367F7006C
:10262000B708010163020702130700002320E60038
:10263000930700002322F60003A7060083A74600A5
:102640003367F700E31207FE03C5050023A0060168
:1026500023A21601E31C05FA6FF01FEB8325C508C2
:10266000130101FB23248104232611042322910456
:1026700023202105232E3103232C4103232A510338
:10268000232861032326710323248103232291033A
:102690002320A103232EB10193078000130405001A
:1026A0006386F516930720006380F506938745FF40
:1026B000130710006376F7009307F0006392F5228A
:1026C00003258408EFF01FC91305040003248104C7
:1026D0008320C10483244104032901048329C10305
:1026E000032A8103832A4103032B0103832BC102A5
:1026F000032C8102832C4102032D0102832DC10191
:10270000130101056FD09F9B03274508937737007E
:1027100063980708EF078000731030000327070055
:1027200083A70700630AF706130510049715000036
:102730009385C5B897F6FFFF9386C68C17F6FFFF03
:102740001306469003A7060083A74600130805005A
:10275000938515003367F700B7080101630207028C
:10276000130700002320E600930700002322F60051
:1027700003A7060083A746003367F700E31207FEAE
:1027800003C5050023A0060123A21601E31C05FAD8
:1027900013053000EFF0DFA913051000EFF05FA97B
:1027A00097150000938545AF1306100497F6FFFFB9
:1027B0009386468517F5FFFF1305C58803A7060016
:1027C00083A74600130E0600938515003367F700B4
:1027D000B70E010163020702930700002320F500F2
:1027E000130800002322050103A7060083A7460063
:1027F0003367F700E31207FE03C6050023A0C601F6
:1028000023A2D601E31C06FA6FF09FF8032B850282
:10281000371C0000974400009384449E171D00005D
:10282000130D4D7EB70C0400974B0000938B8BBCAF
:102830006F00C00123A2870023A08B00B717000000
:10284000330CFC00B7F703006302FC1C9357CC0069
:10285000139437003386840003260600E30006FE47
:102860009387074093972700B307FD0083A70700CE
:1028700013F60704630C06122326F100F3AD0C10C7
:10288000B707C0FFB305FC003716000013050C00A6
:102890002324B100EFF05F87630005028327C100A6
:1028A0008325810093F707086382070A3716000023
:1028B00013050C00EFF0CFF43384840073900D10F7
:1028C00083A70B0023200400E39607F69747000038
:1028D000938787B223A08B0023A087006FF01FF699
:1028E0009305100417160000130606A097E6FFFFD5
:1028F0009386467117E5FFFF1305C57403A706000D
:1029000083A7460013830500130616003367F700FC
:10291000B703010163020702930700002320F500BB
:10292000130800002322050103A7060083A7460021
:102930003367F700E31207FE8345060023A0660015
:1029400023A27600E39C05FA6FF09FE4930710043E
:10295000171600001306069197E6FFFF9386866A16
:1029600097E5FFFF9385056E138907001306160090
:10297000B70901016F004001930700001308000030
:1029800023A0F50023A2050103A7060083A74600A4
:102990003367F700E31207FE8347060023A02601F2
:1029A00023A23601E39207FC6FF09FDE9307100429
:1029B000171600001306C68797E6FFFF9386866406
:1029C00097E5FFFF93850568138A07001306160035
:1029D000B70A01016F0040019307000013080000CF
:1029E00023A0F50023A2050103A7060083A7460044
:1029F0003367F700E31207FE8347060023A0460172
:102A000023A25601E39207FC6FF09FD813050B0039
:102A1000EFF01F82F32740F163920716172600009C
:102A20001306465E9357C600130101F69397A7005D
:102A3000232E1108232C8108971500009385855CAF
:102A400093E7170023A0F500B707002093D6C50031
:102A5000370700809387F70C232EF6FEB3E7E600D6
:102A600073900718F3260018639AD716130405000D
:102A70001347F7FF9307F00197020000938242018A
:102A8000F39252307310073B7390073A97D7BF7F8A
:102A90009387876B73905710F3270034B708C07F74
:102AA000B387170173900714B7B700009387071017
:102AB00073902730B7E701007390073073504030B0
:102AC0009737C07F93870754174700002326F79254
:102AD0009737C07F9387077217470000232CF79022
:102AE00037030800173700001307C751173E0000CF
:102AF000130ECE7093071003930500001303F30326
:102B0000938888001396F50193D61700B366D60014
:102B100033866700B3C7F600330817011316C600E3
:102B2000939757002320C7002322070193F707023A
:102B300013078700B3E7F60093D51500E314EEFC06
:102B400013060009930500001305010097370000E4
:102B500023A4076AEFF08FD0B70700803304F40096
:102B60001305010023228108EFD04FD58320C1092E
:102B7000032481091301010A67800000B7B7B00D73
:102B8000B705080093872765130700009385C5FFE5
:102B900037080080370500406F00C0022FA00600F4
:102BA0001316F70193D61700B366D600B3C7D70044
:102BB0009397E7013376F5001357170093870600C4
:102BC0003367E600B3F6B70013F61700B3860601C5
:102BD000E31606FC03A006006FF09FFC93051004AB
:102BE000170600001306067397E6FFFF93868641DB
:102BF00017E5FFFF1305054503A7060083A7460059
:102C000013880500130616003367F700B7080101A3
:102C100063020702130700002320E500930700006A
:102C20002322F50003A7060083A746003367F700B9
:102C3000E31207FE8345060023A0060123A2160126
:102C4000E39C05FA13053000EFF08FDE678000008B
:102C5000930000001301000033872000930E000052
:102C6000930120006316D74D93001000130110004C
:102C700033872000930E200093013000631AD74B56
:102C8000930030001301700033872000930EA000E2
:102C900093014000631ED749930000003781FFFF76
:102CA00033872000B78EFFFF930150006312D7498E
:102CB000B70000801301000033872000B70E0080AA
:102CC000930160006316D747B70000803781FFFF8C
:102CD00033872000B78EFF7F93017000631AD745BA
:102CE00093000000378100001301F1FF33872000BB
:102CF000B78E0000938EFEFF93018000631AD743C6
:102D0000B70000809380F0FF13010000338720009C
:102D1000B70E0080938EFEFF93019000631AD74197
:102D2000B70000809380F0FF378100001301F1FFAE
:102D300033872000B78E0080938EEEFF9301A000B2
:102D40006318D73FB7000080378100001301F1FFFF
:102D500033872000B78E0080938EFEFF9301B00072
:102D60006318D73DB70000809380F0FF3781FFFFE5
:102D700033872000B78EFF7F938EFEFF9301C00044
:102D80006318D73B930000001301F0FF3387200046
:102D9000930EF0FF9301D000631CD7399300F0FF2E
:102DA0001301100033872000930E00009301E00010
:102DB0006310D7399300F0FF1301F0FF3387200031
:102DC000930EE0FF9301F0006314D73793001000D7
:102DD000370100801301F1FF33872000B70E008018
:102DE000930100016316D7359300D0001301B000A2
:102DF000B3802000930E800193011001639AD033B9
:102E00009300E0001301B00033812000930E900185
:102E100093012001631ED1319300D000B3801000D4
:102E2000930EA001930130016394D031130200008E
:102E30009300D0001301B000338720001303070074
:102E40001302120093022000E31452FE930E80013D
:102E500093014001631ED32D130200009300E00094
:102E60001301B00033872000130000001303070094
:102E70001302120093022000E31252FE930E9001FF
:102E8000930150016316D32B130200009300F0004E
:102E90001301B0003387200013000000130000006E
:102EA000130307001302120093022000E31052FEE6
:102EB000930EA00193016001631CD327130200004D
:102EC0009300D0001301B0003387200013021200DA
:102ED00093022000E31652FE930E800193017001CD
:102EE0006318D725130200009300E0001301B0001F
:102EF0001300000033872000130212009302200009
:102F0000E31452FE930E9001930180016312D723C4
:102F1000130200009300F0001301B0001300000042
:102F200013000000338720001302120093022000D8
:102F3000E31252FE930EA00193019001631AD71F72
:102F4000130200009300D000130000001301B00032
:102F5000338720001302120093022000E31452FE74
:102F6000930E80019301A0016314D71D130200008A
:102F70009300E000130000001301B00013000000F4
:102F8000338720001302120093022000E31252FE46
:102F9000930E90019301B001631CD7191302000036
:102FA0009300F00013000000130000001301B000B4
:102FB000338720001302120093022000E31252FE16
:102FC000930EA0019301C0016314D71713020000F0
:102FD0001301B0009300D0003387200013021200C9
:102FE00093022000E31652FE930E80019301D0015C
:102FF0006310D715130200001301B0009300E00026
:1030000013000000338720001302120093022000F7
:10301000E31452FE930E90019301E001631AD7115D
:10302000130200001301B0009300F0001300000031
:1030300013000000338720001302120093022000C7
:10304000E31252FE930EA0019301F0016312D70F19
:10305000130200001301B000130000009300D00021
:10306000338720001302120093022000E31452FE63
:10307000930E800193010002631CD70B1302000022
:103080001301B000130000009300E00013000000E3
:10309000338720001302120093022000E31252FE35
:1030A000930E9001930110026314D70913020000DC
:1030B0001301B00013000000130000009300F000A3
:1030C000338720001302120093022000E31252FE05
:1030D000930EA00193012002631CD7059300F0001A
:1030E00033011000930EF000930130026312D105FA
:1030F0009300000233810000930E0002930140020E
:103100006318D103B3000000930E00009301500236
:103110006390D003930000011301E001338020008D
:10312000930E0000930160026314D001631A300013
:10313000139511006300050013651500730000006E
:0C3140001305100073000000731000C0A5
:10314C00417373657274696F6E206661696C656436
:10315C003A2061646472203E3D202831554C203C5D
:10316C003C203132292026262061646472203C20C8
:10317C003633202A202831554C203C3C2031322932
:10318C000A000000417373657274696F6E2066618A
:10319C00696C65643A20212870745B315D5B6164F5
:1031AC0064722F2831554C203C3C203132295D2053
:1031BC00262030783038302920262620636175731C
:1031CC0065203D3D203078660A0000004173736530
:1031DC007274696F6E206661696C65643A206E6FFB
:1031EC0064650A00417373657274696F6E20666161
:1031FC00696C65643A20757365725F6D6170706996
:10320C006E675B616464722F2831554C203C3C2006
:10321C003132295D2E61646472203D3D20300A00FC
:10322C00417373657274696F6E206661696C656455
:10323C003A2070745B315D5B616464722F28315588
:10324C004C203C3C203132295D2026203078303413
:10325C00300A0000417373657274696F6E20666189
:10326C00696C65643A2070745B315D5B6164647297
:10327C002F2831554C203C3C203132295D20262012
:10328C0030783038300A0000417373657274696F9E
:10329C006E206661696C65643A2074662D3E6570BB
:1032AC006320252034203D3D20300A004173736596
:1032BC007274696F6E206661696C65643A202122B4
:1032CC00696C6C6567616C20696E7374727563747C
:1032DC00696F6E220A000000417373657274696F26
:1032EC006E206661696C65643A202122756E657882
:1032FC0070656374656420657863657074696F6E5E
:10330C00220A0000417373657274696F6E206661E6
:10331C00696C65643A202122756E737570706F72DA
:10332C007465642073617470206D6F6465220A008B
:040000058000000077
:00000001FF
